:100000000C9466000C9483000C9483000C94830081
:100010000C9483000C9483000C9483000C94450290
:100020000C9483000C9483000C9483000C94830044
:100030000C9483000C9483000C9483000C94830034
:100040000C94FB010C9483000C9483000C948300AB
:100050000C9483000C9483000C9483000C94830014
:100060000C9483000C9483000000000024002700FF
:100070002A0000000000250028002B0000000000DE
:1000800023002600290004040404040404040202DA
:100090000202020203030303030302020301020438
:1000A00008102040800102040810200102040810FA
:1000B0002040804000000009000302000004050801
:1000C00000000000000000000000000011241FBE1E
:1000D000CFEFD8E0DEBFCDBF11E0A0E0B1E0EAEAAB
:1000E000F8E002C005900D92A030B107D9F721E0E9
:1000F000A0E0B1E001C01D92AD30B207E1F70E946F
:1001000087020C9453040C940000843081F028F48E
:100110008230E9F08330F9F00895883071F0893049
:1001200091F08530B9F4809180008F7D03C080917B
:1001300080008F778093800008958091B0008F7742
:100140008093B00008958091B0008F7DF9CF84B581
:100150008F7784BD089584B58F7DFBCFCF93DF93D8
:10016000282F30E0F901EC54FF4F8491F901E35658
:10017000FF4FD491F901EA57FF4FC491CC23A1F06E
:1001800081110E948500EC2FF0E0EE0FFF1FE45874
:10019000FF4FA591B491EC91ED2381E090E009F43B
:1001A00080E0DF91CF91089580E090E0FACF1F9337
:1001B000CF93DF93282F30E0F901EC54FF4F849167
:1001C000F901E356FF4FD491F901EA57FF4FC4916B
:1001D000CC23A9F0162F81110E948500EC2FF0E0AE
:1001E000EE0FFF1FEE58FF4FA591B4918FB7F89413
:1001F000EC91111108C0D095DE23DC938FBFDF9105
:10020000CF911F910895DE2BF8CFCF93DF9390E02D
:10021000FC01E356FF4F24918A579F4FFC018491C4
:100220008823D1F090E0880F991FFC01E859FF4F17
:10023000A591B491FC01EE58FF4FC591D491611185
:100240000EC09FB7F8948C91E22FE0958E238C938B
:100250002881E223E8839FBFDF91CF9108958FB774
:10026000F894EC91E22BEC938FBFF6CF883020F01E
:100270008D3008F48DE08E508770806480937C0010
:1002800080917A00806480937A0080917A0086FD64
:10029000FCCF809178009091790008953FB7F89451
:1002A0008091090190910A01A0910B01B0910C017C
:1002B00026B5A89B05C02F3F19F00196A11DB11DC1
:1002C0003FBFBA2FA92F982F8827BC01CD01620FFD
:1002D000711D811D911D42E0660F771F881F991FB8
:1002E0004A95D1F708958F929F92AF92BF92CF9285
:1002F000DF92EF92FF926B017C010E944E014B0155
:100300005C01C114D104E104F104B9F00E944E0172
:10031000681979098A099B09683E7340810591052E
:1003200080F321E0C21AD108E108F10888EE880EB6
:1003300083E0981EA11CB11CE4CFFF90EF90DF90EA
:10034000CF90BF90AF909F908F900895E0E8F0E03D
:1003500080818F77808361E089E00E94D70062E32B
:1003600070E080E090E00E94730160E081E00E9414
:10037000D700109201011092000187E08093B10034
:100380000895CF93DF93C0E8D0E088818F7788838A
:1003900060E089E00E94D70064E670E080E090E0D1
:1003A0000E94730161E089E00E94D7008881806823
:1003B0008883E1E8F0E0808181608083DF91CF91E4
:1003C0000895CF93DF93EC0161E080E00E94D700B5
:1003D000BE0190E080E00E94730161E081E00E9434
:1003E000D70062E370E080E090E00E947301DF914B
:1003F000CF910C94C1011F920F920FB60F9211244E
:100400002F933F938F939F93AF93BF938091050159
:1004100090910601A0910701B0910801309104016B
:1004200023E0230F2D3768F126E8230F0296A11D44
:10043000B11D209304018093050190930601A093C0
:100440000701B09308018091090190910A01A091E0
:100450000B01B0910C010196A11DB11D8093090102
:1004600090930A01A0930B01B0930C01BF91AF913F
:100470009F918F913F912F910F900FBE0F901F90E2
:1004800018950196A11DB11DD4CF1F920F920FB6E2
:100490000F9211242F933F934F935F936F937F930A
:1004A0008F939F93AF93BF93EF93FF93809100013E
:1004B0009091010101969093010180930001209198
:1004C0000001309101018091020190910301821796
:1004D000930760F410920101109200011092B10094
:1004E0001092B20060E080E00E94D700FF91EF918F
:1004F000BF91AF919F918F917F916F915F914F913C
:100500003F912F910F900FBE0F901F9018957894E8
:1005100084B5836084BD85B5836085BD80916E00A0
:10052000816080936E00C2E0C09381008091810061
:100530008160809381008091800081608093800041
:100540008091B10084608093B1008091B00081609F
:100550008093B00087E880937A001092C10060E039
:1005600082E00E94050160E085E00E94050160E0F4
:1005700086E00E94050161E089E00E94050161E0DA
:1005800089E00E94D70061E080E00E94050161E0FF
:1005900081E00E94050110928000109281008BE0A2
:1005A00091E0909387008093860080918000826024
:1005B00080938000809181008861809381001092F7
:1005C000B0001092B100C093B0008CE98093B300EA
:1005D000C0937000789488248A9483E0982EA12C8C
:1005E000B12C81E10E9436018C0180E10E9436012C
:1005F00028EB3BE0DC010E944C04A50194010E9421
:10060000FC03309303012093020183E10E94360131
:1006100020E23EE4DC010E944C04A50194010E940A
:10062000FC0369017A0182E10E94360120E23EE486
:10063000DC010E944C04A50194010E94FC032901E5
:100640003A01209086003090870086E00E943601B3
:100650009101DC010E944C04A50194010E94FC035D
:10066000309389002093880085EF481681E0580672
:1006700040F495EFC91691E0D906B0F5CEE6D0E08A
:100680000BC085EFC81681E0D80680F561E08AE0EE
:100690000E94D700C7E7D1E082E00E94AE00892B1C
:1006A00081F5D1112EC020E23EE4D8010E944C0415
:1006B000A50194010E94FC03C901CE36C9F0C037E0
:1006C00009F450C0C436E9F40E94E101C701B60143
:1006D000882799270E9473010E94A60182E00E9448
:1006E000AE00892BD9F30DC0C4E6C9CFC0E7C7CF90
:1006F0000E94E10182E00E94AE00892BD9F30E94A2
:10070000A60186E00E94AE00892B91F480918000C2
:100710008F778093800060E089E00E94D70086E0B8
:100720000E94AE00892BD9F361E089E00E94D700D6
:1007300085E00E94AE00892B69F461E080E00E94B0
:10074000D70085E00E94AE00892BD9F360E080E0FD
:100750000E94D70080E090E0892B09F442CF0E94EC
:1007600000003FCF0E94E101EE24FF24C701B60143
:100770000E9473016624772482E00E94AE00892BD8
:1007800009F0BDCF809180008F778093800061E079
:1007900089E00E94D70062E370E080E090E00E9470
:1007A000730160E081E00E94D70082E00E94AE0009
:1007B000892B09F0A4CFC301B2010E94730182E02A
:1007C0000E94AE00892B09F09ACF61E081E00E947F
:1007D000D70062E370E080E090E00E9473010E9425
:1007E000C10182E00E94AE00892B09F088CFC701C9
:1007F000B6010E947301C0CF052E97FB1EF4009432
:100800000E94130457FD07D00E941B0407FC03D06D
:100810004EF40C94130450954095309521953F4F1C
:100820004F4F5F4F089590958095709561957F4FDC
:100830008F4F9F4F0895A1E21A2EAA1BBB1BFD01EB
:100840000DC0AA1FBB1FEE1FFF1FA217B307E407AF
:10085000F50720F0A21BB30BE40BF50B661F771F07
:10086000881F991F1A9469F76095709580959095E7
:100870009B01AC01BD01CF010895A29FB001B39FC0
:10088000C001A39F700D811D1124911DB29F700D99
:10089000811D1124911D08950E943D04B7FF089504
:0A08A000821B930B0895F894FFCF1C
:00000001FF
